:040000000134013492
:20003400758171D2AFD28C1204BF12001B80FB0581740A75F000C0E0C0F0740275F000C095
:20005400E0C0F01207B115811581158115815480C5F05400C5F078FE122705F645F07003F6
:20007400020095E61227377BFF12272E12283845F0700302009274FF75F0FF02009A02007B
:2000940045740175F000158122120043740A75F000C0E0C0F0740075F000C0E0C0F074014F
:2000B40075F000C0E0C0F01207DA7FFA122711221200437BFF7CFF12283845F07003020039
:2000D400DD74FF75F0FF020146740A75F000C0E0C0F0740075F000C0E0C0F0743875F000A2
:2000F400C0E0C0F01207DA7FFA122711120043740A75F000C0E0C0F0740075F000C0E0C025
:20011400F0740C75F000C0E0C0F01207DA7FFA12271112009D740075F000C0E0C0F07400A4
:2001340075F000C0E0C0F012014715811581158115812212004378FB122705E61227379036
:200154000209022740740A75F000C0E0C0F0740075F000C0E0C0F078F5122705E624801274
:200174002737C0E0C0F01207DA7FFA12271102021D740A75F000C0E0C0F0740075F000C01A
:20019400E0C0F078F5122705E624C0122737C0E0C0F01207DA7FFA12271102021D740A75BC
:2001B400F000C0E0C0F0740075F000C0E0C0F078F5122705E62494122737C0E0C0F01207A0
:2001D400DA7FFA12271102021D740A75F000C0E0C0F0740075F000C0E0C0F078F512270546
:2001F400E624D4122737C0E0C0F01207DA7FFA12271102021DDD010300B10102008501015A
:20021400005901000000001D02220581740078FE122705F678FE122705E61818181886010A
:2002340008860275F00012272789828A83E4931227377B0012272E12284145F0700302024D
:20025400A4800B78FE122705E604F61480C6120043740A75F000C0E0C0F0740175F000C04B
:20027400E0C0F078FA122705E618181818860108860275F00012272789828A83E493122740
:2002940037C0E0C0F01207DA7FFA12271102025778FA122705E60886F0158122120043741D
:2002B4000A75F000C0E0C0F0740175F000C0E0C0F078F7122705E6122737C0E0C0F01207D5
:2002D400DA7FFA122711227F0812271178F3122705E60886F07B007C0012281845F070037C
:2002F40002030A740075F00079F712270A122727742DF702031A740075F00079F712270AAC
:20031400122727742BF778F3122705E60886F078FD122705F608A6F078F3122705E6088662
:20033400F07B007C0012281845F0700302036878FD122705E60886F012281178F312270550
:20035400F608A6F018E60886F01227FE18F608A6F0122807740175F00079F712270A12278F
:200374002778F3122705E60886F07BE87C031227842430C5F03400C5F0F718E60886F07BB6
:20039400E87C0312277D78FD122705F608A6F0740275F00079F712270A12272778FD122749
:2003B40005E60886F07B647C001227842430C5F03400C5F0F778F3122705E60886F07B64D3
:2003D4007C0012277D78FD122705F608A6F0740375F00079F712270A12272778FD122705EE
:2003F400E60886F07B0A7C001227842430C5F03400C5F0F7740475F00079F712270A122715
:200414002778FD122705E60886F07B0A7C0012277D2430C5F03400C5F0F7740075F0007998
:20043400F712270A122727E7122737C0E0C0F01202B015811581740175F00079F712270AEA
:20045400122727E7122737C0E0C0F01202B015811581740275F00079F712270A122727E7BC
:20047400122737C0E0C0F01202B015811581740375F00079F712270A122727E7122737C0B2
:20049400E0C0F01202B015811581740475F00079F712270A122727E7122737C0E0C0F0121F
:2004B40002B0158115817FF8022720758E03E5A84481F5A8E5884401F5887400F53A74004F
:2004D400F56C740C75F000C0E0C0F0740075F000C0E0C0F0E53A122737C0E0C0F01207DA77
:2004F4007FFA1227117400F511747075F017F55D85F05E746475F000F55385F05479637A82
:2005140000E98AF0C0E0C0F0746475F000C0E0C0F012250A15811581158115811218691249
:2005340000C474E075F02BC0E0C0F012021E15811581740075F000C0E0C0F0740175F0004E
:20055400C0E0C0F0120147158115811581158174E975F02BC0E0C0F012021E158115817476
:200574008075F025C0E0C0F012253D1581158179A07A28E98AF0C0E0C0F0122560158115BD
:2005940081120FB41210AB7400F508121016120F93120E6C1209A4120D97120BCF120C4775
:2005B400120C8412117D1213A812155312196E121747121A05121A2E121AEC121D5112213F
:1D05D4002812097B1213E112144B12147D12076D120E4312221B12228F0205982276
:07000300C0D0C0E00205F1CE
:2005F100C0F0C083C082C000C001C002C003C004C005C006C007120625D007D006D005D00A
:2006110004D003D002D001D000D082D083D0F0D0E0D0D032E59054BFF590740875F000C0EA
:20063100E0C0F0740275F000C0E0C0F01207B11581158115811581F53D85F03E740875F006
:2006510000C0E0C0F0740175F000C0E0C0F01207B11581158115811581F53F85F040E53FE0
:200671008540F05410C5F05400C5F0F53BE53F8540F05420C5F05400C5F0F53CE53F85403D
:20069100F0540FC5F05400C5F0F53F85F040E53F8540F07B087C001227DFF53F85F040E591
:2006B1003D853EF0453FC5F04540C5F0F53D85F03EE53B60030206DAE53D853EF07BFF7CB1
:2006D100FF122769F53D85F03EE53C70030206EB740F75F027F53D85F03EE53A122737C3B6
:2006F10033C5F033C5F079437A00122727E53D853EF0F709A7F0E53A04F53A14E53A54033B
:20071100F53A740C75F000C0E0C0F0740075F000C0E0C0F0E53A122737C0E0C0F01207DA69
:200731007FFA122711740A75F000C0E0C0F012259C15811581E5904440F590E53A122737A6
:200751007B0012272E12283845F0700302076CE59054BFF590E5114480F51122E51675F0C8
:20077100007B627C0012283845F07003020795795B7A2BE98AF0C0E0C0F0122560158115E9
:2007910081120FB42278FB122705E6F513E513A2E09290A2E19291A2E29292A2E39293227B
:2007B10078F9122705E6122737C0E0C0F01207961581158178FB122705E60886F0C0E0C083
:2007D100F01225B9158115812278F7122705E6122737C0E0C0F01207961581158178F91229
:2007F1002705E60886F0C0E0C0F008E6122737C0E0C0F01225DA15811581158115812212BD
:2008110025FA74D075F000C0E0C0F012260F15811581740775F000C0E0C0F012260F15812F
:200831001581749075F000C0E0C0F012260F15811581122607221225FA74D075F000C0E00A
:20085100C0F012260F15811581740075F000C0E0C0F012260F158115811226071225FA74E4
:20087100D175F000C0E0C0F012260F158115817400F5717400F515E51575F0007B067C00BA
:2008910012284B45F070030208C08008E51504F5151480E3E515794B7A0075F0001227274C
:2008B100C001C002122639D007D000F602089D7401F571E515794B7A0075F000122727C057
:2008D10001C002122639D007D000F6122607221225FA74D075F000C0E0C0F012260F1581CE
:2008F1001581740075F000C0E0C0F012260F15811581740075F000C0E0C0F012260F1581AF
:200911001581743075F000C0E0C0F012260F15811581741275F000C0E0C0F012260F15814C
:200931001581740375F000C0E0C0F012260F15811581742575F000C0E0C0F012260F158146
:200951001581740775F000C0E0C0F012260F15811581740075F000C0E0C0F012260F158147
:2009710015811226072212084722E51675F0007B757C0012283845F070030209A379DA7A8B
:200991002AE98AF0C0E0C0F012256015811581120FB422E51675F0007B747C00122838452D
:2009B100F07003020A4F74F175F02BC0E0C0F012256015811581120B06F50D743A75F00028
:2009D100C0E0C0F012257415811581120B06F50C743A75F000C0E0C0F01225741581158181
:2009F100120B06F50A1225FA74D075F000C0E0C0F012260F15811581740075F000C0E0C0EE
:200A1100F012260F15811581E50A75F000C0E0C0F012260F15811581E50C75F000C0E0C095
:200A3100F012260F15811581E50D75F000C0E0C0F012260F15811581122607120FB4227F73
:200A510009122711740075F00078FD122705F608A6F012258CC0E0C0F01225741581158128
:200A710078FC122705F67B0D7C0012284145F07003020AB8801678FD122705E60886F01213
:200A910027FE18F608A6F012280780C678FD122705E60886F079F612270A12272778FC123E
:200AB1002705E6F7020A8778FD122705E60886F079F612270A1227277400F778FD12270542
:200AD100E60886F07B007C0012283845F07003020AEB74FF75F0FF020B0179F612270AE919
:200AF1008AF0C0E0C0F012266D15811581020B017FF702272005810581058105810581746B
:200B11000075F00078FD122705F608A6F078FD122705E60886F07B027C0012281845F07011
:200B310003020B78801678FD122705E60886F01227FE18F608A6F012280780D178FD12274C
:200B510005E60886F079FA12270A122727C001C00212258CC0E0C0F012257415811581D0C8
:200B710007D000F6020B3778FD122705E60886F079FA12270A1227277400F7740075F000E2
:200B910079FA12270A122727E7C394301227377B0412272E1227DFC0E0C0F0740175F00028
:200BB10079F812270A122727E7C39430D004D0034BC5F04CC5F01227377FFB022720E516CC
:200BD10075F0007B697C0012283845F07003020C46741075F02CC0E0C0F01225601581152A
:200BF10081740075F000C0E0C0F012079615811581740475F000C0E0C0F0120A507B647C6B
:200C110000122769C0E0C0F01225E81581158115811581740475F000C0E0C0F01225C81519
:200C3100811581F55D85F05EE55D855EF0F55B85F05C120FB422E51154087003020C83E5FF
:200C51005B855CF0122807F55B85F05C1227FEE55B855CF07B007C0012285245F070030280
:200C71000C83E55D855EF0F55B85F05CE5114404F51122E51714F51704E51775F0007B003C
:200C91007C0012285245F07003020D967464F517120847740075F000C0E0C0F012079615BC
:200CB100811581740275F000794B7A00122727C001C002740075F000C0E0C0F01225B915E2
:200CD100811581D007D00086037C0012283845F0602B740175F000794B7A00122727C001D5
:200CF100C002740175F000C0E0C0F01225B915811581D007D00086037C0012283845F07018
:200D110003020D25E5114408F511742C75F001F55385F054740275F000794B7A00122727B3
:200D3100C001C002740275F000C0E0C0F01225B915811581D007D00086037C001228384575
:200D5100F0602B740175F000794B7A00122727C001C002740375F000C0E0C0F01225B915DB
:200D7100811581D007D00086037C0012283845F07003020D96E51154F7F511746475F0005C
:200D9100F55385F05422E51675F0007B647C0012283845F07003020E42742875F02CC0E01B
:200DB100C0F012256015811581120B06F50E742D75F000C0E0C0F012257415811581120B3F
:200DD10006F50F742D75F000C0E0C0F012257415811581120B06F5101225FA74D075F000C9
:200DF100C0E0C0F012260F15811581740475F000C0E0C0F012260F15811581E50E75F00027
:200E1100C0E0C0F012260F15811581E50F75F000C0E0C0F012260F15811581E51075F00088
:200E3100C0E0C0F012260F15811581122607120FB422E51675F0007B0D7C0012283845F09D
:200E51007003020E6B79A07A28E98AF0C0E0C0F012256015811581120FB422E51675F0000B
:200E71007B2F7C0012283845F07003020F92120847744775F02CC0E0C0F0740475F000792B
:200E91004B7A00122727E775F000C0E0C0F0740575F000794B7A00122727E775F000C0E018
:200EB100C0F0740675F000794B7A00122727E775F000C0E0C0F0740475F0001222C67FF80A
:200ED100122711745875F02CC0E0C0F0740275F000794B7A00122727E775F000C0E0C0F0F5
:200EF100740175F000794B7A00122727E775F000C0E0C0F0740075F000794B7A0012272756
:200F1100E775F000C0E0C0F0740475F0001222C67FF8122711121082746875F02CC0E0C01B
:200F3100F0740075F00079437A00122727E70987F0C0E0C0F0740275F00079437A00122740
:200F510027E70987F0C0E0C0F0740475F00079437A00122727E70987F0C0E0C0F074067589
:200F7100F00079437A00122727E70987F0C0E0C0F0740575F0001222C67FF6122711120F6B
:200F9100B422E59854017003020FAF12258CC0E0C0F012257415811581F516020FB374FF39
:200FB100F5162279E57A28E98AF0C0E0C0F0122560158115812205810581740075F00078FE
:200FD100FD122705F608A6F078FD122705E60886F078F9122705860308860412281845F0C9
:200FF1007003021011801678FD122705E60886F01227FE18F608A6F012280780CB020FF825
:20101100158115812212101D12105722E559855AF01227FEF55985F05A122807E559855AD8
:20103100F0AB53AC5412285B45F07003021056740075F000F55985F05AE5114440F511C2D4
:20105100977405F51422E51154407003021081E51414F51404E51475F0007B007C0012280B
:201071003845F07003021081D297E51154BFF51122C297E5904440F590E511548075F0004C
:201091007B007C0012283845F070030210A202108AE511547FF511D29722308DFDC28D4338
:2010B1008CDC2205810581740175F00079637A00122727E775F00078FD122705F608A6F066
:2010D10018E60886F07B087C001227DF18F608A6F0740075F00079637A0012272778FD12AA
:2010F1002705E60886F047158115812274012563F563E43564F564E43565F565221210FD76
:20111100740275F00079637A00122727E775F000C0E0C0F0120796158115811210B42212AC
:2011310010FD1210FD740275F00079637A00122727E775F000C0E0C0F0120796158115816A
:201151001210B42278FB122705E675F0007B047C001227EDF62430C5F03400C5F02278FBEC
:20117100122705E6540F243012273722E51154047003021366121082120847121130C0E0BD
:20119100C0F0E5578558F0C0E0C0F01225E8158115811581158112110EC0E0C0F074047550
:2011B100F000794B7A00122727E775F000C0E0C0F01225DA158115811581158112110EC09A
:2011D100E0C0F0740575F000794B7A00122727E775F000C0E0C0F01225DA15811581158183
:2011F100158112110EC0E0C0F0740675F000794B7A00122727E775F000C0E0C0F01225DA9D
:20121100158115811581158112110EC0E0C0F0740275F000794B7A00122727E775F000C05F
:20123100E0C0F01225DA158115811581158112110EC0E0C0F0740175F000794B7A001227D2
:2012510027E775F000C0E0C0F01225DA158115811581158112110EC0E0C0F0740075F000F7
:20127100794B7A00122727E775F000C0E0C0F01225DA1581158115811581121130C0E0C007
:20129100F0740075F00079437A00122727E70987F0C0E0C0F01225E81581158115811581B0
:2012B100121130C0E0C0F0740275F00079437A00122727E70987F0C0E0C0F01225E815819D
:2012D100158115811581121130C0E0C0F0740475F00079437A00122727E70987F0C0E0C05E
:2012F100F01225E81581158115811581121130C0E0C0F0740675F00079437A00122727E777
:201311000987F0C0E0C0F01225E81581158115811581E51154FBF511E5578558F01227FEEA
:20133100F55785F058121367740075F000C0E0C0F012079615811581740675F000C0E0C0B4
:20135100F0E5578558F0C0E0C0F01225E8158115811581158122E5578558F07B887C1312ED
:20137100285B45F070030213A7E51154F7F511746475F000F55385F054743C75F000C0E02B
:20139100C0F074FF75F0FFC0E0C0F01225DA158115811581158122E51675F0007B727C0011
:2013B10012283845F070030213E0747575F02CC0E0C0F0E5578558F0C0E0C0F0740275F00F
:2013D100001222C61581158115811581120FB422740E75F000C0E0C0F0740075F000C0E003
:2013F100C0F01207B115811581158115817BFF7C0012284145F0600EE511540175F0007BCB
:20141100007C0012283845F07003021446E5114401F511740E75F000C0E0C0F0740075F078
:2014310000C0E0C0F01207B11581158115811581F53702144A74FFF53722740E75F000C035
:20145100E0C0F0740075F000C0E0C0F01207B115811581158115817BFF7C0012283845F003
:20147100700302147CE51154FEF51122E53775F0007BFF7C0012284145F07003021552E5FE
:201491003775F00090153E022740E56C04F56C14021552E5116402F511E51154EFF511126D
:2014B100009D740075F000C0E0C0F0740175F000C0E0C0F012014715811581158115817405
:2014D1008B75F02CC0E0C0F012021E15811581E511540270030214FC742A75F000C0E0C0FD
:2014F100F01202B01581158102153512009D12218F740075F000C0E0C0F0740075F000C07C
:20151100E0C0F01201471581158115811581749375F02CC0E0C0F012021E15811581E5113C
:201531004410F5110215520215520215523B15EF003815DF00A414BF009B147F00000052A3
:201551001522E51675F0007B737C0012283845F070030216EA740075F000C0E0C0F012071B
:201571009615811581749C75F02CC0E0C0F0740075F000C0E0C0F01225B915811581C0E0C2
:20159100C0F0740175F000C0E0C0F01225B915811581C0E0C0F0740375F0001222C67FFAA5
:2015B100122711740075F000C0E0C0F0120B06C0E0C0F01225DA1581158115811581743A1D
:2015D10075F000C0E0C0F012257415811581740175F000C0E0C0F0120B06C0E0C0F012259A
:2015F100DA158115811581158174AF75F02CC0E0C0F0740275F000C0E0C0F01225B91581F3
:201611001581C0E0C0F0740375F000C0E0C0F01225B915811581C0E0C0F0740375F000124D
:2016310022C67FFA122711740275F000C0E0C0F0120B06C0E0C0F01225DA1581158115817D
:201651001581743A75F000C0E0C0F012257415811581740375F000C0E0C0F0120B06C0E0BA
:20167100C0F01225DA158115811581158174C275F02CC0E0C0F0740075F000C0E0C0F012EE
:2016910025B915811581C0E0C0F0740175F000C0E0C0F01225B915811581C0E0C0F07402D3
:2016B10075F000C0E0C0F01225B915811581C0E0C0F0740375F000C0E0C0F01225B9158146
:2016D1001581C0E0C0F0740575F0001222C67FF61227111216EB120FB422740075F000C0D9
:2016F100E0C0F01225B9158115817B997C0012283845F07003021729743C75F000C0E0C0CC
:20171100F0740175F000C0E0C0F01225DA1581158115811581021746743C75F000C0E0C061
:20173100F074FF75F0FFC0E0C0F01225DA158115811581158122E51675F0007B3D7C001250
:20175100283845F07003021868740075F000C0E0C0F01207961581158174D875F02CC0E06D
:20177100C0F0740075F000C0E0C0F01225B915811581C0E0C0F0740175F000C0E0C0F012D7
:2017910025B915811581C0E0C0F0740375F0001222C67FFA12271174EA75F02CC0E0C0F006
:2017B100740275F000C0E0C0F01225B915811581C0E0C0F0740375F000C0E0C0F01225B965
:2017D10015811581C0E0C0F0740375F0001222C67FFA12271174FC75F02CC0E0C0F074041A
:2017F10075F000C0E0C0F01225C8158115817B647C00122784C0E0C0F0740275F000122281
:20181100C61581158115811581743C75F000C0E0C0F01225B9158115817B017C00122838AE
:2018310045F07003021850741A75F02DC0E0C0F0740175F0001222C6158115810218657422
:201851002375F02DC0E0C0F0740175F0001222C615811581120FB422740075F000C0E0C042
:20187100F012079615811581740475F000C0E0C0F01225C815811581F55D85F05EE55D8548
:201891005EF0F55B85F05C740675F000C0E0C0F01225C815811581F55785F05879697A00F9
:2018B100E98AF0C0E0C0F0742E75F000C0E0C0F012250A158115811581158179667A00E932
:2018D1008AF0C0E0C0F0E5578558F0C0E0C0F012250A158115811581158179667A00E98A6F
:2018F100F0C0E0C0F079697A00E98AF0C0E0C0F012245C158115811581158179667A00E95C
:201911008AF0C0E0C0F0746475F000C0E0C0F012250A1581158115811581796D7A00E98AF3
:20193100F0C0E0C0F079667A00E98AF0C0E0C0F012241B158115811581158179637A00E962
:201951008AF0C0E0C0F0796D7A00E98AF0C0E0C0F01224CD158115811581158122E51675AC
:20197100F0007B6E7C0012283845F07003021A04742A75F02DC0E0C0F01225601581158184
:2019910012258C7B797C0012283845F07003021A01E51154F7F511740075F000F55785F0EB
:2019B10058740075F000C0E0C0F012079615811581740675F000C0E0C0F0740075F000C0F2
:2019D100E0C0F01225E8158115811581158179637A00E98AF0C0E0C0F0746475F000C0E009
:2019F100C0F012250A1581158115811581121FBE120FB422E51675F0007B3F7C001228389F
:201A110045F07003021A2D79E97A28E98AF0C0E0C0F012256015811581120FB422E51675E3
:201A3100F0007B637C0012283845F07003021AEB120847743D75F02DC0E0C0F0740475F059
:201A510000794B7A00122727E775F000C0E0C0F0740575F000794B7A00122727E775F00073
:201A7100C0E0C0F0740675F000794B7A00122727E775F000C0E0C0F0740475F0001222C615
:201A91007FF8122711744E75F02DC0E0C0F0740275F000794B7A00122727E775F000C0E06B
:201AB100C0F0740175F000794B7A00122727E775F000C0E0C0F0740075F000794B7A001228
:201AD1002727E775F000C0E0C0F0740475F0001222C67FF8122711120FB422E51675F0001C
:201AF1007B617C0012283845F07003021D5012209279667A00E98AF0C0E0C0F0740175F04A
:201B110000C0E0C0F012250A158115811581158179637A00E98AF0C0E0C0F079667A00E980
:201B31008AF0C0E0C0F012242E158115811581158179667A00E98AF0C0E0C0F079637A00AC
:201B5100E98AF0C0E0C0F01224CD158115811581158179637A00E98AF0C0E0C0F074647510
:201B7100F000C0E0C0F012250A1581158115811581740075F000F56185F062E5618562F058
:201B9100AB57AC5812284B45F07003021D4D8012E5618562F01227FEF56185F06212280741
:201BB10080D9740D75F000C0E0C0F0121FAC15811581740A75F000C0E0C0F0121FAC1581D6
:201BD1001581121130C0E0C0F01225C815811581745E75F02DC0E0C0F0E5618562F0C0E01F
:201BF100C0F0740275F0001222C61581158115811581746275F02DC0E0C0F012110EC0E06E
:201C1100C0F01225B915811581C0E0C0F012110EC0E0C0F01225B915811581C0E0C0F01298
:201C3100110EC0E0C0F01225B915811581C0E0C0F0740475F0001222C67FF812271174723A
:201C510075F02DC0E0C0F012110EC0E0C0F01225B915811581C0E0C0F012110EC0E0C0F023
:201C71001225B915811581C0E0C0F012110EC0E0C0F01225B915811581C0E0C0F07404750D
:201C9100F0001222C67FF8122711748275F02DC0E0C0F0121130C0E0C0F01225C815811563
:201CB10081C0E0C0F0740275F0001222C61581158115811581748675F02DC0E0C0F0121116
:201CD10030C0E0C0F01225C815811581C0E0C0F0740275F0001222C61581158115811581CB
:201CF100748A75F02DC0E0C0F0121130C0E0C0F01225C815811581C0E0C0F0740275F000FA
:201D11001222C61581158115811581748E75F02DC0E0C0F0121130C0E0C0F01225C8158144
:201D31001581C0E0C0F0740275F0001222C61581158115811581121F72021BA1120FB42227
:201D5100E51675F0007B787C0012283845F07003021F7112209279667A00E98AF0C0E0C017
:201D7100F0740175F000C0E0C0F012250A158115811581158179637A00E98AF0C0E0C0F096
:201D910079667A00E98AF0C0E0C0F012242E158115811581158179667A00E98AF0C0E0C04E
:201DB100F079637A00E98AF0C0E0C0F01224CD158115811581158179637A00E98AF0C0E065
:201DD100C0F0746475F000C0E0C0F012250A1581158115811581740075F000F56185F06216
:201DF100E5618562F0AB57AC5812284B45F07003021F6E8012E5618562F01227FEF5618532
:201E1100F06212280780D9740D75F000C0E0C0F0121FAC15811581740A75F000C0E0C0F053
:201E3100121FAC15811581121130C0E0C0F01225C815811581749275F02DC0E0C0F0E5618C
:201E51008562F0C0E0C0F0740275F0001222C6158115811581158112110EC0E0C0F0122565
:201E7100B91581158112110EC0E0C0F01225B91581158112110EC0E0C0F01225B9158115B3
:201E91008112110EC0E0C0F01225B91581158112110EC0E0C0F01225B91581158112110E45
:201EB100C0E0C0F01225B915811581749675F02DC0E0C0F0121130C0E0C0F01225C8158181
:201ED1001581C0E0C0F0740275F0001222C61581158115811581749A75F02DC0E0C0F012DC
:201EF1001130C0E0C0F01225C815811581C0E0C0F0740275F0001222C61581158115811519
:201F110081749E75F02DC0E0C0F0121130C0E0C0F01225C815811581C0E0C0F0740275F042
:201F3100001222C6158115811581158174A275F02DC0E0C0F0121130C0E0C0F01225C8158F
:201F5100811581C0E0C0F0740275F0001222C61581158115811581121F72021E06120FB43E
:201F71002205811226B17B137C0012283845F07003021FA978FE122705E61227377B111229
:201F9100272E12284145F07003021FA91226B178FE122705F6021F8515812278FB1227054C
:201FB100E6F5133099FDC299E513F5992274A675F02DC0E0C0F01225601581158179187A8F
:201FD10000E98AF0C0E0C0F0741E75F000C0E0C0F01226C31581158115811581740075F0CA
:201FF10000C0E0C0F012079615811581740075F000F56185F062E5618562F079187A001265
:202011002727E775F0007B007C0012284145F0700302206C8012E5618562F01227FEF56131
:2020310085F06212280780CEE5618562F02408C5F03400C5F0C0E0C0F0E5618562F0791844
:202051007A00122727E775F000C0E0C0F01225DA1581158115811581022027E5618562F02A
:202071002408C5F03400C5F0C0E0C0F0740075F000C0E0C0F01225DA1581158115811581A3
:20209100220581740D75F000C0E0C0F0121FAC15811581740A75F000C0E0C0F0121FAC1523
:2020B100811581740075F000C0E0C0F012079615811581740075F000F56185F062E5618523
:2020D10062F02408C5F03400C5F0C0E0C0F01225B91581158178FE122705F67B007C0012B4
:2020F100284145F070030221258012E5618562F01227FEF56185F06212280780C078FE125A
:202111002705E6122737C0E0C0F0122574158115810220FC158122740075F000C0E0C0F006
:2021310012079615811581743C75F000C0E0C0F01225B9158115817B017C0012283845F093
:20215100700302218EE5B0540875F0007B007C0012283845F0700302217EE5114408F511FA
:20217100742C75F001F55385F05402218EE51154F7F511746475F000F55385F0542274005B
:2021910075F000C0E0C0F012079615811581743C75F000C0E0C0F01225B9158115817B01A1
:2021B1007C0012283845F070030221ED740775F000C0E0C0F0740175F000C0E0C0F01201FB
:2021D100471581158115811581744D75F000C0E0C0F01202B01581158102221A740775F0CB
:2021F10000C0E0C0F0740175F000C0E0C0F01201471581158115811581744175F000C0E0E8
:20221100C0F01202B01581158122E5115402700302228E121082740075F000C0E0C0F07439
:202231000075F000C0E0C0F01201471581158115811581E56C5403F56CE56C243175F00012
:20225100C0E0C0F01202B015811581742075F000C0E0C0F01202B015811581E56C75F0003E
:20227100C333C5F033C5F079437A00122727E70987F0C0E0C0F01202DB1581158122E5113A
:20229100541070030222C5740075F000C0E0C0F0740175F000C0E0C0F01201471581158194
:2022B10015811581E5578558F0C0E0C0F01202DB158115812223F42581F886820886830875
:2022D100E4FEFF93700122B42555A3E493B42D06430780A3E493B4300343074024D0B40AB0
:2022F10000500CCE75F00AA42EFEA3E49380EDE493B46413E60886F030F708430720122804
:202311000EA6F018F68003B4750543070A801CB478054307108014B46F0B430708800C121C
:20233100257AA3809BB462624307027A00C004C005C006C007AB0753031F7C00E60886F0D4
:202351001227ACA6F018F6EDD007D006D005D0042430B43A0040022407C0E00AE645F070BC
:20237100CCA902EF30E506742D12257A0A1223FCD0E012257AD9F90808EF30E7A5EAC39E05
:2023910050A0742012257A0A80F3B4630BAA011223FCE612257A80DFB4732BC082C0838629
:2023B100820886837A00E4936004A30A80F886831886821223FCE493A3600512257A80F6FF
:2023D100D083D08280B1B4691986017A00E76004090A80F91223FC8601E7609B12257A09B4
:2023F10080F7F97A011223FCE980A8EE601B8FF020F716C002EAC39E500D742030F60274F0
:202411003012257A0A80EED002221225277A04C3E637F60809DAF9E4F5F092E0221225270D
:202431007A04C3E697F60809DAF980EB12251FC37A04E633F608DAFA80DD12251F7A04C80D
:202451002AC8C318E613F6DAFA80CC122527AB00A8817F0412271108AC001224D01225336C
:20247100A80312244E5007786DA90412241EA8031224DC600CA804122440A8041224DC7066
:20249100DFA803796D1224D07FFC022720122527AB00AC011225337D21C3A803122441DD71
:2024B100028033786D122441786DA9041224EB20E7E7786DA904122431D380DE1225277A57
:2024D10004E7F60908DAFA2212251F7A0475F000E6700308DAFA221225277A04E82AF8E9A4
:2024F1002AF9181987F0E6B5F006DAF6E4F5F02274FF40F904F5F00422E58124FBF98700F4
:2025110012253587000909E7F60809E7F622E58124FBF8860022E58124FBF88601181886D9
:202531000022786D7A04760008DAFB2278FB1227058603088604748075F0701227AC1228DC
:202551000E758921F58DF58B7588597598522278FB1227058682088683E493602D12257AE5
:20257100A380F678FB122705E63099FDC299F599B40A17740D80F2E430980C3098FDC2984C
:20259100E599B40D02740A75F0002278FB1227058603088604BB0004BC00012279E5A3D9A0
:2025B100FD1BBBFFF01C80F478FB1227058682088683E075F0002278FB1227058682088640
:2025D10083E0F5F0A3E0C5F02278F9122705868208868308E6F02278F9122705868208863B
:2025F1008308E608F0A3E6F022D29512265FC295122665C29422C29512265FD2952278FB72
:20261100122705E67F0830E704D2958002C29512265F23C294DFEFD29512265F30950012F0
:202631002665C294122665227F087400D29512265FA29533C294DFF6C0E0D295E571B4004A
:2026510002C29512265FC294D0E075F00022D2943094FD22000022000000002278FB1227B3
:20267100058601E4FBFCFFE709B42D030FE709C39430B40A005012FA740A75F000122769EA
:202691002AFBE5F03400FC80E4EB8CF0DF0302280E2278FB122705E63099FDC299F5992290
:2026B10074FFF5F030980A3098FDC298E59975F0002278FB122705860418188601E4FD12D6
:2026D100258CB408028003B47F16ED60F21D740812257A742012257A740812257A1980DF3B
:2026F10012257AF724F36006090DEDB504D1E4F7F5F0ED22C82581C822C92581C97A00221C
:20271100D083D082CF2581F581CFC082C08322CF2581F581CF2229F9E5F03AFA227C00CB32
:2027310030E7011CCB2275F00030E70215F022FDE493A3FEE493A3FF4E7009E493FE7401E3
:2027510093FF800BE493A3B5050BE493B5F0068F838E82E473A380D8FEEBA4FD8EF0ECA43E
:20277100FCEB8EF0A4C5F02C2DC5F0221227AC8EF0ED22C0F0C0E0E5F06C5480FF8CF030D8
:20279100F707EB12280EACF0FBD0E0D0F030F70312280EBF80051227AC8062C002C001AA46
:2027B100F0F97E007D007F11C3E933F9EA33FADF08F5F0E9D001D00222ED33FDEE33FEC32C
:2027D100ED9BF5F0EE9C40E0ADF0FED380DBBB000122C333C5F033C5F0DBF722BB000122C5
:2027F100C3C5F013C5F013DBF7221227FE04700205F02212280714B4FF0215F0221228074B
:20281100F4C5F0F4C5F02212286B4029801E12286B40227017801E12286B40107017800C53
:2028310012286B5010800512287F6009E4F5F02212287F60F7E4F5F0042212287F40F68082
:20285100EB12287F40EF70E480EB12287F40DD70E480D912287F50DD80D2C39BC5F09C204B
:20287100E70720D207C345F02220D2F9D322C5F0C39C7003E5F09B22FBE493CB22FCE4937B
:20289100FB740193CC22FAE493F9740193CA220A0A4D696E694C4F474745522056332E3070
:2028B10020284329203230303320572E5349524943484F544520446570742E6F662041709E
:2028D100706C6965642050687973696373204B4D49544C000A3E3E000A0A48454C50204D05
:2028F100454E55202020202020202020202020202020200A2F2072656164206F6E63652005
:202911002020202020202020202020202020200A742054494D4520736574202020202020CD
:20293100202020202020202020200A642044415445207365742020202020202020202020CE
:2029510020202020200A6320436C6F636B20646973706C61792020202020202020202020D7
:2029710020202020200A732053544152542F53544F50207265636F7264696E672074696DBF
:2029910065202020202020202020202020202020200A6920496E74657276616C2020202069
:2029B1002020202020202020202020200A3D2073657474696E6720706172616D6574657240
:2029D10073202020202020202020202020202020200A72206E756D626572206F6620726562
:2029F100636F7264202020202020202020202020202020200A62207465726D696E616C2016
:202A1100636F6E6E656374696F6E202020202020202020202020202020200A6E204E6577B3
:202A3100207265636F7264202020202020202020202020202020200A6120414C4C2072658B
:202A510061643A2073616D706C65207265616C2D74696D6520616E642064617461202020B7
:202A7100202020202020202020202020200A78205265616420416C6C3A2073616D706C6572
:202A910020616E642064617461202020202020202020202020202020200A752041626F75F2
:202AB10074204D696E694C4F474745522056332E302020202020202020202020202020203D
:202AD100200A3F2068656C70000A4D696E694C4F474745522077617320646573696E6765F2
:202AF1006420627920572E5349524943484F5445203238204A756E65203230303320202096
:202B110020202020202020202020202020200A55524C3A207777772E6B6D69746C2E6163E7
:202B31002E74682F7E6B7377696368697420656D61696C3A206B73776963686974406B6D67
:202B510069746C2E61632E7468000A2031202020203220202020332020202034202020202B
:202B710035202020203620202020372020202038202020203920202031302020313120208E
:202B9100313220202020202020202020202020202020202020200A494E312B20494E312D2F
:202BB10020494E322B20494E322D20494E332B20494E332D20494E342B20494E342D202D33
:202BD1003556202B35562020305620202B56004D696E694C4F47470045522056332E3000A8
:202BF1000A656E7465722063757272656E742074696D652048483A4D4D3A5353203E000ADE
:202C110020696E74657276616C20312D36303020736563203E20000A656E74657220637511
:202C31007272656E7420646174652044442D4D4D2D5952203E000A253032782D25303278C0
:202C51002D253032782000253032783A253032783A2530327820002025642025642025648B
:202C7100202564000A2575207265636F72647320617661696C61626C650078302E316D5659
:202C910020005265636F72643D20000A535441525420253032783A25303278203E000A539C
:202CB100544F502020253032783A25303278203E000A20253032783A253032782025303231
:202CD100783A25303278000A20535441525420253032783A25303278000A2053544F502092
:202CF10020253032783A25303278000A2053414D504C494E4720494E54455256414C2873C6
:202D1100656329203D202575000A204D414E55414C000A204155544F000A204E6577207269
:202D310065636F72643F28592F4E29000A253032782D253032782D25303278200025303207
:202D5100783A253032783A2530327820002025640020253032782D253032782D2530327838
:202D71000020253032783A253032783A25303278002025640020256400202564002025640D
:202D91000020256400202564002025640020256400202564000A3C2D2D20456E74657220F7
:202DB1006465736372697074696F6E207465787420286D6178203330206368617261637472
:092DD100657273292D2D3E0A00E4
:00000001FF
